S10E2000CF400016209C87CE30028EDB
S110200B304827056A000820F6CE2115CDC7
S111201830008E21172706180A307020F516A6
S1072026202A20FE4A
S1052115304252
S111202A34B7751B9ECC00017C3042CC304292
S11020387C3000CC00027C3022CC30427C95
S10C20453006CC301A7C3008CCC2
S10C204E301A7C3004CC30067C0D
S11120573002CC00341620A1201FCC2090169D
S111206520DDCC00006C1ECC20891620DDECA2
S11120731EC300016C1EEC1E8C03202DEC20FD
S10B2081DFCC0000B757303D2D
S111208941206C696E650048656C6C6F2057D1
S10820976F726C64008F
S108209C1D0016073DC4
S11120A13B34B775EC027C00C0C60C7B00C358
S10920AFB757301B823D0F
S11120B53B34B775FC3046270CE603C10A26FF
S11120C306CC000D1620B51F00C480FB180DBE
S10F20D10300C7E60387B757301B823DAD
S11120DD3B34B7751B9ECC00006C1E2016ED24
S11120EB02E640871620B5EC1EC300016C1EF1
S11120F9EC02C300016C02ED02E74026E4CCC9
S1112107000A1620B5CC0001B757301B823DEC
S9032000DC
